:100000000AC03BC01895189518951895189518951D
:100010001895189518958FED8DBFC0ECE0EC4E2E1D
:10002000DD275D2EEEE7F0E0A0E6B0E088278D93B7
:100030003197E9F766248FE087BB8BEF81BB80E7C0
:1000400088BB84E082BB939A84E690E082D3939845
:1000500084E690E07ED3939A84E690E07AD39398F6
:1000600078948BB780648BBFC398C298C198C098AE
:1000700085B7806385BF8895F7CFEAE0F0E0AEE60C
:1000800091E0A1D300916E000E3C08F004C085B74A
:10009000806385BF8895E3E1F0E0AEE691E093D31D
:1000A00000916E000E3C08F004C085B7806385BFE8
:1000B0008895C39AC29AC19AC09A80E080936A00D8
:1000C00080E080936900ACE653D3A1E653D380E08F
:1000D00080936500ACE6E1D2BF98AFE69C9197FFB4
:1000E00004C0B7990EC09F779C93B79B0AC088E263
:1000F0009F9399272ED39F91B79B03C090689C93A1
:10010000B9D2C39AC0988CE080936000BC98AFE6E7
:100110009C9196FF04C0B49B0EC09F7B9C93B499A6
:100120000AC088E29F93992714D39F91B49903C082
:1001300090649C931DD18AE080936000BD98AFE6E7
:100140009C9195FF04C0B59B0EC09F7D9C93B59973
:100150000AC088E29F939927FCD29F91B59903C06A
:1001600090629C9305D18BE080936000BE98AFE6CF
:100170009C9194FF04C0B69B0EC09F7E9C93B69941
:100180000AC088E29F939927E4D29F91B69903C051
:1001900090619C93EDD0C09AC19889E080936000F3
:1001A000BC98AFE69C9196FF04C0B49B0EC09F7BA9
:1001B0009C93B4990AC088E29F939927CAD29F91D1
:1001C000B49903C090649C93D3D088E0809360007E
:1001D000BD98AFE69C9195FF04C0B59B0EC09F7D76
:1001E0009C93B5990AC088E29F939927B2D29F91B8
:1001F000B59903C090629C93BBD087E08093600068
:10020000BE98AFE69C9194FF04C0B69B0EC09F7E43
:100210009C93B6990AC088E29F9399279AD29F919E
:10022000B69903C090619C93A3D0C19AC29886E00E
:1002300080936000BC98AFE69C9196FF04C0B49B8D
:100240000EC09F7B9C93B4990AC088E29F93992724
:1002500080D29F91B49903C090649C9389D085E02B
:1002600080936000BD98AFE69C9195FF04C0B59B5C
:100270000EC09F7D9C93B5990AC088E29F939927F1
:1002800068D29F91B59903C090629C9371D084E02D
:1002900080936000BE98AFE69C9194FF04C0B69B2B
:1002A0000EC09F7E9C93B6990AC088E29F939927BF
:1002B00050D29F91B69903C090619C9359D0C29A35
:1002C000C39883E080936000BC98AFE69C9196FF52
:1002D00004C0B49B0EC09F7B9C93B4990AC088E273
:1002E0009F93992736D29F91B49903C090649C93B1
:1002F0003FD082E080936000BD98AFE69C9195FF6F
:1003000004C0B59B0EC09F7D9C93B5990AC088E23E
:100310009F9399271ED29F91B59903C090629C9399
:1003200027D081E080936000BE98AFE69C9194FF57
:1003300004C0B69B0EC09F7E9C93B6990AC088E20B
:100340009F93992706D29F91B69903C090619C9381
:100350000FD081E090E0FDD1ACE60D911C91083802
:1003600053E1150710F009F001C0B4CE18950895B7
:10037000ACE6FED1939A84E690E0EBD1939884E6C4
:1003800090E0E7D1A6E30C9104FB81E00EF480E05D
:100390008F93A6E30C9105FB81E00EF480E09F9122
:1003A000892B8F93A6E30C9106FB81E00EF480E08D
:1003B0009F91892B882309F401C0E4CF0091690043
:1003C000013009F015C08091600080936A000091AF
:1003D0006A00043010F009F001C001C0E2C0A9E6D3
:1003E0008C918F5F8C9380E080936500F7D00895A7
:1003F00000916900023009F001C051C0009169000C
:10040000033009F001C06AC0009160000B3009F0B0
:1004100008C0A9E68C918F5F8C9380E08093650083
:100420000895009160000C3009F038C048EE53E0A8
:1004300060E070E0A1E60D911D912D913C91A5D158
:100440000CF401C002C0ADC029C0E2E0F0E0A4E1BC
:1004500094E0B9D19AD109F002C0E4C01FC0E6E02F
:10046000F0E0A4E194E0AFD190D109F002C0DAC08D
:1004700015C0EBE0F0E0A4E194E0A5D186D109F04D
:1004800002C0D0C00BC0EFE0F0E0A4E194E09BD14B
:100490007CD109F002C0C6C001C083C056C0009123
:1004A00060000C3009F019C0E2E0F0E0A4E194E053
:1004B0008AD1A1E60D911D912D913C9166D109F44F
:1004C00001C06FC08BD0A1E655D180E0809365005C
:1004D000A9E68C918F5F8C93089537C000916000DE
:1004E0000C3009F032C000916A00013009F007C0F9
:1004F000E2E0F0E0A1E694E07BE754D11FC00230D7
:1005000009F007C0E6E0F0E0A1E694E07BE74AD11D
:1005100015C0033009F007C0EBE0F0E0A1E694E07D
:100520007BE740D10BC0043009F007C0EFE0F0E0FA
:10053000A1E694E07BE736D101C033C04FD08CEE0A
:1005400093E1ACE68D939C930895A5E68C918F5F23
:100550008C9300916500063010F009F001C001C0D5
:1005600020C0A1E60D911D912D913C914AE050E0F3
:1005700060E070E09FD0A1E60D931D932D933D9315
:10058000A1E60D911D912D913C91A0E64C9155272E
:1005900066277727F5D0A1E60D931D932D933D9304
:1005A0000895ABE68C918F5F8C9389E08093670010
:1005B0008FE5809368001AD000916B00033009F03A
:1005C00007C0ECE3F0E070D080E080936B0006D0D1
:1005D0008CEE93E1ACE68D939C93089582E080933A
:1005E000670088EC8093680001D0089581E08093D3
:1005F00066004091670000916600041710F009F052
:1006000010C0939AA8E68C919927A3D09398A8E656
:100610008C9199279ED0A6E68C918F5F8C9308F4DD
:10062000E8CF089580E080936B00A1E6A3D0D6DFE9
:1006300084EF91E08ED0949AE1E0F0E035D0949888
:10064000E1E0F0E031D080916E00815080936E0047
:10065000EAE0F0E0AEE691E07BE7A4D0E3E1F0E091
:10066000AEE691E07BE79ED08CEE93E1ACE68D9315
:100670009C930895E4E0F0E017D0B79901C00CC056
:10068000E2E0F0E002ED14E020E030E0A0E1BB2782
:1006900094E07BE787D0A2DF0895ED91FC91EF5FB6
:1006A000FF4FFC93EE93089588EE93E052D031977C
:1006B000D9F7089522D006D000FC01D0089528D0A3
:1006C00030D00895842F952FA62FB72F4427552774
:1006D00066277727F1E2889409C020F4480F591F54
:1006E0006A1F7B1F76956795579547953795279590
:1006F00017950795FA9589F708950024E89477FFF0
:1007000002C006D0689400F809D010F801240895BA
:1007100012D04F5F5F4F6F4F7F4F0895E89437FFC0
:10072000089500951095209530950F5F1F4F2F4F1E
:100730003F4F689408954095509560957095089541
:100740003197F1F70895689462F80895E89462F893
:100750000895EF93FF93EE27E82BE92B31F0E8EEB5
:10076000F3E03197F1F70197D1F7FF91EF910895F9
:1007700082E001C084E099279D938A95E9F7089566
:10078000040F151F261F371F089504171507260786
:1007900037070895E199FECFEEBB3196089591E0B9
:1007A00001C092E07B3751F47FB7F894F3DF8D916D
:1007B0008DBBE29AE19A9A95C9F77FBF7727089592
:1007C00091E001C092E0E6DFE09A8DB38D939A95B7
:0407D000D1F70895C0
:00000001FF
